:100000000C949A000C94B5000C94B5000C94B500B7
:100010000C94B5000C94B0050C9469060C940F0672
:100020000C943C060C9483050C94B5000C941105BB
:100030000C94B5000C94B5000C94B5000C94B5006C
:100040000C94B5000C94B5000C94B5000C94B5005C
:1000500030313233343536373839414243444546FE
:1000600000000000000300060008000A00001F0056
:100070000000001F00001F101010101F00001F18AC
:100080001818181F00001F1C1C1C1C1F00001F1E1E
:100090001E1E1E1F00001F1F1F1F1F1F0003070F14
:1000A0001F0F070300001F1F1F1F1F1F001B1B1B0D
:1000B0001B1B1B1B00181C1E1F1E1C180000040409
:1000C0000E0E1F1F00001F1F0E0E04040000000074
:1000D0000000000000000E1915130E0000000E15A0
:1000E00015150E0000000E1315190E0000000E115C
:1000F0001F110E00002D2057656C636F6D65207415
:100100006F20746865204545323831204C6162208B
:100110002333204C43442054657374202D00436FD7
:100120006E74726173743A202564200054696D65A1
:10013000723A000011241FBECFE5D8E0DEBFCDBF6C
:1001400010E0A0E6B0E0ECECF2E202C005900D9207
:10015000A036B107D9F710E0A0E6B0E001C01D92CB
:10016000AC38B107E1F70C940B080C9400009093A5
:100170006100809360000895CF93DF93EC01892B99
:1001800061F08881882349F08991E0916000F091C5
:100190006100099588818823B9F7DF91CF9108958F
:1001A000EF92FF921F93CF93DF93EC01892B71F1B4
:1001B00010E077276115710559F08881811121962A
:1001C0001F5F812F992787FD909586179707ACF3BE
:1001D00010E0E42EFF24E114F104C1F088818823AB
:1001E00079F02196E0916000F091610009951F5F20
:1001F000812F992787FD90958E159F057CF306C06A
:10020000E0916000F091610080E2F0CFDF91CF914A
:100210001F91FF90EF900895CF93DF93EC0100972B
:1002200079F0FC0121968491882351F0E0916000DF
:10023000F09161000995FE01219684918823B1F720
:10024000DF91CF910895E0916000F09161008DE021
:100250000995E0916000F09161008AE009950895A8
:10026000E82FFF27EF70F070E05BFF4F8491E09183
:100270006000F0916100099508951F93182F8295F1
:100280008F700E943001812F0E9430011F910895CC
:100290000F931F938C01812F99270E943D01802F7E
:1002A0000E943D011F910F910895EF92FF920F93CD
:1002B0001F937B018C01C801AA27BB270E9448011C
:1002C000C7010E9448011F910F91FF90EF90089580
:1002D0002F923F924F925F926F927F928F929F9256
:1002E000AF92BF92CF92DF92EF92FF920F931F9344
:1002F000CF93DF93CDB7DEB7A2970FB6F894DEBFEA
:100300000FBECDBF69A3442E2AA337014801442361
:1003100009F483C017FF81C0EE24FF248701E6188B
:10032000F7080809190999A1692F772767FD7095C2
:1003300061507040442011F061507040562E18A258
:100340002FE1222E312C2C0E3D1EA82EBB24A7FC03
:10035000B094CB2CDB2CC801B701A60195010E94FB
:10036000F110DC01CB01FC01E05BFF4F84918F8F2A
:10037000C801B701A60195010E94F11079018A0117
:100380005A94EFEF5E1609F1E114F104010511052D
:1003900009F43EC0C801B701A60195010E94F11001
:1003A000DC01CB01FC01E05BFF4F8491F101829302
:1003B0001F01C801B701A60195010E94F110790142
:1003C0008A015A949FEF5916F9F6442031F097FEAE
:1003D00016C08DE2F10182931F0159A05A94FFEFDC
:1003E0005F16F1F0F10181911F01E0916000F09141
:1003F000610009955A94FFEF5F16A1F711C016141A
:1004000017041804190414F48BE2E4CF80E2E2CF5D
:10041000F1018AA182931F01D4CF8401730183CF9C
:10042000A2960FB6F894DEBF0FBECDBFDF91CF917D
:100430001F910F91FF90EF90DF90CF90BF90AF9002
:100440009F908F907F906F905F904F903F902F90F4
:1004500008955F926F927F928F929F92AF92BF9218
:10046000CF92DF92EF92FF920F931F93CF93DF9380
:10047000982E7A018B0155240F2EF0E0AF2EF0E07C
:10048000BF2EF0E8CF2EFFE3DF2EF02DC52D20E0AC
:1004900030E040E050E0C801B7010E94A80D882379
:1004A0000CF4C1E020E030E040E050E0C801B701CA
:1004B0000E942C0D18160CF0AAC0852CA6019501DF
:1004C000C801B7010E94FB0BDC01CB0120E030E04A
:1004D00040E251E4BC01CD010E94A80D87FD0EC091
:1004E00020E030E040E251E4C601B5010E94790A03
:1004F0005B016C0183948EE0881500F7CC2309F42E
:1005000080C0E0916000F09161008DE2099588243F
:10051000692C772467FC7094161417040CF07CC0C7
:10052000A6019501C801B7010E94FB0BDC01CB01BC
:10053000BC01CD010E949E08DC01CB01982E8529CB
:10054000C82FDD2720E030E040E85FE3C601B501B9
:100550000E94EE0C882319F0CD2B09F44CC03FEF1C
:10056000532E892D805DE0916000F0916100099526
:1005700020E030E040E85FE3C601B5010E94EE0CE8
:10058000882391F1892D9927AA2797FDA095BA2F45
:10059000BC01CD010E94E60DDC01CB01A601950155
:1005A000BC01CD010E94790ADC01CB019C01AD01A7
:1005B000C801B7010E94440ADC01CB017C018D0116
:1005C00020E030E040E251E4C601B5010E94FB0B9F
:1005D000DC01CB015C016D018394882D9927861580
:1005E00097050CF49DCF18C0E0916000F091610078
:1005F0008EE20995C7CFE0916000F091610080E242
:10060000B6CFE0916000F09161008BE27FCF17FBE5
:10061000109517F9109551CFDF91CF911F910F9140
:10062000FF90EF90DF90CF90BF90AF909F908F9012
:100630007F906F905F9008957F928F929F92AF927C
:10064000BF92CF92DF92EF92FF920F931F93CF93BF
:10065000DF93CDB7DEB77888C988DA8873E1A72E33
:10066000B12CAC0EBD1E772009F482C0F6010894AF
:10067000C11CD11C8491853249F0882309F47CC0C7
:10068000E0916000F09161000995EDCF772009F4C9
:100690006BC0F6010894C11CD11C8491282F33270C
:1006A00027FD30952436310509F456C0253631052D
:1006B00054F42336310521F7F50122E030E0A20E93
:1006C000B31E8081DDCF28373105D1F640E1E42E1D
:1006D000F12C4701F50122E030E0A20EB31E0081AB
:1006E00011818436D1F0C801B7010E94DD10FB01F1
:1006F000E05BFF4F8491E0916000F091610009950B
:10070000C801B7010E94DD108C01C701B4010E942D
:10071000DD107B01672B39F7A6CF17FF09C01095B5
:1007200001951F4FE0916000F09161008DE2099505
:1007300032E0E316F104B8F20E151F05A0F6C7016A
:100740006AE070E00E94DD107B016230710558F2B2
:1007500006171707A0F3C7CF6AE0862E912C50E149
:10076000E52E57E2F52EB6CFF60181916F0196CFB7
:10077000F60181916F017FCF80E090E0DF91CF9112
:100780001F910F91FF90EF90DF90CF90BF90AF90AF
:100790009F908F907F900895E0916000F0916100AC
:1007A00009950895039665E070E00E94DD109B01B5
:1007B00044275527DA01C90163E0880F991FAA1F52
:1007C000BB1F6A95D1F7821B930BA40BB50B20E0DE
:1007D00030E02817390728F42F5F3F4F28173907D3
:1007E000D8F30895CF93C0E08C2F0E943D04CF5FD3
:1007F000C730D0F30E9403040E940D040E94160427
:100800007894CF91089582E00E94200412BE89B7A7
:10081000816089BF0E949004089583E00E942604AD
:100820001DBC1CBC89B7846089BF089583E00E9409
:100830002C0414BC89B7806489BF0E94AC0408955D
:10084000982F83B7887F892B83BF0895982F8EB503
:10085000887F892B8EBD0895982F85B5887F892B39
:1008600085BD0895873040F4E82FFF27EE0FFF1F66
:10087000EE59FF4F608371830895873040F4E82F6D
:10088000FF27EE0FFF1FEE59FF4F108211820895D0
:10089000EF92FF920F931F93AC0183B7E82FFF27CE
:1008A000EE0FFF1FEF59FF4F249180E091E07A0196
:1008B0000027112702C0880F991F2A95E2F79C0193
:1008C0004427552760E070E880E790E00E9413110C
:1008D000C801B7010E94BE10DC01CB01BC01CD01F3
:1008E00028EE33E040E050E00E941311109288009F
:1008F0001092890010928A0010928B0080918800DB
:1009000090918900A0918A00B0918B008217930783
:10091000A407B50798F31F910F91FF90EF900895EA
:10092000109278001092790010927A0010927B0059
:100930001092840010928500109286001092870019
:1009400008958091780090917900A0917A00B091FB
:100950007B00BC01CD0108951092800010928100AF
:10096000109282001092830010927C0010927D0001
:1009700010927E0010927F000895809180009091E7
:100980008100A0918200B0918300BC01CD01089547
:10099000893059F08A3031F08FB58D7F8FBD8FB59A
:1009A000816008C08FB58260F9CF8FB582608FBD3E
:1009B0008FB58E7F8FBD8EB588608EBD8FB58068F8
:1009C0008FBD8FB58F7B8FBD8FB580628FBD8FB58B
:1009D0008F7E8FBD1BBC1ABC19BC18BC08958FB587
:1009E0008D7F8FBD8FB58E7F8FBD8EB5877F8EBD7E
:1009F0008FB58F778FBD8FB58F7B8FBD8FB58F7D77
:100A00008FBD8FB58F7E8FBD08959C01892F99274B
:100A10008BBD2ABD08959C01892F992789BD28BDCA
:100A200008951F920F920FB60F9211242F933F93A8
:100A30004F935F936F937F938F939F93AF93BF93E6
:100A4000EF93FF938091780090917900A0917A00C4
:100A5000B0917B000196A11DB11D80937800909309
:100A60007900A0937A00B0937B00809178009091F8
:100A70007900A0917A00B0917B000097A105B105A3
:100A800099F48091840090918500A0918600B091A6
:100A900087000196A11DB11D80938400909385006D
:100AA000A0938600B0938700809188009091890080
:100AB000A0918A00B0918B000196A11DB11D809379
:100AC000880090938900A0938A00B0938B00809156
:100AD000620090916300892B29F0E0916200F0910F
:100AE00063000995FF91EF91BF91AF919F918F9115
:100AF0007F916F915F914F913F912F910F900FBE1A
:100B00000F901F9018951F920F920FB60F921124FD
:100B10002F933F934F935F936F937F938F939F9305
:100B2000AF93BF93EF93FF93809164009091650022
:100B3000892B29F0E0916400F09165000995FF91FF
:100B4000EF91BF91AF919F918F917F916F915F9145
:100B50004F913F912F910F900FBE0F901F901895BE
:100B60001F920F920FB60F9211242F933F934F9322
:100B70005F936F937F938F939F93AF93BF93EF9305
:100B8000FF938091800090918100A0918200B091AC
:100B900083000196A11DB11D809380009093810078
:100BA000A0938200B0938300809180009091810097
:100BB000A0918200B09183000097A105B10599F43E
:100BC00080917C0090917D00A0917E00B0917F008B
:100BD0000196A11DB11D80937C0090937D00A09390
:100BE0007E00B0937F0080916C0090916D00892B06
:100BF00029F0E0916C00F0916D000995FF91EF9163
:100C0000BF91AF919F918F917F916F915F914F9124
:100C10003F912F910F900FBE0F901F9018951F922C
:100C20000F920FB60F9211242F933F934F935F9320
:100C30006F937F938F939F93AF93BF93EF93FF93A4
:100C40008091660090916700892B29F0E091660001
:100C5000F09167000995FF91EF91BF91AF919F913E
:100C60008F917F916F915F914F913F912F910F9055
:100C70000FBE0F901F9018951F920F920FB60F92F4
:100C800011242F933F934F935F936F937F938F9391
:100C90009F93AF93BF93EF93FF93809168009091E0
:100CA0006900892B29F0E0916800F09169000995AD
:100CB000FF91EF91BF91AF919F918F917F916F9134
:100CC0005F914F913F912F910F900FBE0F901F900A
:100CD00018951F920F920FB60F9211242F933F93E6
:100CE0004F935F936F937F938F939F93AF93BF9334
:100CF000EF93FF9380916A0090916B00892B29F00C
:100D0000E0916A00F0916B000995FF91EF91BF911E
:100D1000AF919F918F917F916F915F914F913F9193
:100D20002F910F900FBE0F901F9018959498939845
:100D300092988C9A8B9A8A9A1ABA8FEF8BBB0895E5
:100D400094981ABA8FEF8BBB939A929A0000000086
:100D5000CF9B0CC092980000000000000000929A07
:100D60000000000000000000CF99F4CF9298089591
:100D70001F93182F0E94A00694989398929A8FEF31
:100D80008ABB1BBB000000000000000092981ABA4A
:100D90008BBB1F9108950E94A0061ABA8FEF8BBBE0
:100DA0009498939A929A000000000000000089B382
:100DB0009298992708951F93182F0E94A006949A3D
:100DC0009398929A8FEF8ABB1BBB00000000000033
:100DD000000092981ABA8BBB1F9108950E94A0063A
:100DE0001ABA8FEF8BBB949A939A929A00000000E4
:100DF0000000000089B39298992708950E949606F2
:100E000088E30E94B80681E00E94B80686E00E944E
:100E1000B8068CE00E94B80682E00E94B80680E81E
:100E20000E94B80640E0642F8DE690E00E946B07B8
:100E300041E0642F8DE690E00E946B0742E0642F52
:100E40008DE690E00E946B0743E0642F8DE690E012
:100E50000E946B0744E0642F8DE690E00E946B07D0
:100E600045E0642F8DE690E00E946B0746E0642F1A
:100E70008DE690E00E946B0747E0642F8DE690E0DE
:100E80000E946B07089582E00E94B806089581E0F1
:100E90000E94B8060895382F862F99278130910532
:100EA00099F08230910564F08230910531F0232F62
:100EB0002C5A039759F0232F09C0232F2C5E06C00C
:100EC000232F892B19F0F7CF232F205C2068822F46
:100ED0000E94B8060895CF92DF92EF92FF920F938F
:100EE0001F93CF93DF936C01062F142F0E94CB0624
:100EF000F82E8FE7F822110F110F110F000F000FBE
:100F0000000FEE24C0E0D0E0812F8E0D80640E949F
:100F1000B806F601E00FF11DEC0FFD1F84910E9451
:100F2000DB062196E39487E08E1570F780E8F82AB7
:100F30008F2D0E94B806DF91CF911F910F91FF90E6
:100F4000EF90DF90CF900895FF920F931F93CF9370
:100F50008C01F62E892B61F0C0E0C61748F4F80129
:100F6000EC0FF11D80810E94DB06CF5FCF15B8F337
:100F7000CF911F910F91FF9008950F931F93CF93DF
:100F8000DF939C01042F842F9927289FA001299F7C
:100F9000500D389F500D1124CA019A01220F331FA2
:100FA000220F331F280F391F280F391FC9010E9434
:100FB000DD10EB0110E01017D8F486E0189F9001C7
:100FC0001124C9010596C817D90780F4C217D307A1
:100FD00038F480E00E94DB061F5F101770F308C032
:100FE000CE0166E070E00E94DD10F4CF85E0F2CF24
:100FF000DF91CF911F910F9108951ABA17BA14BAC1
:1010000011BA8FEF8BBB88BB85BB82BB85BB84BB12
:101010008D9A95980895CFE5D8E0DEBFCDBF0E94A8
:10102000FD070E94F20384E690E00E9448040E94BB
:10103000FE068BED96E00E94B70088E00E94C8048F
:1010400087E390E00E9405058FB58F7D8FBD8FB53A
:101050008F7E8FBD84E690E00E94480460E0862F7A
:101060000E944B0785EF90E00E940C010E943C0813
:1010700080E090E00C946511AF92BF92CF92DF9226
:10108000EF92FF920F931F93CF93AA24C7E361E0DF
:1010900080E00E944B07CC2EDD242FEFE22EF12CB6
:1010A000C7018C199D099F938F938EE191E09F93C7
:1010B0008F9391E0B92EBF920E941C036B2D8EE09E
:1010C0000E944B070F900F900F900F900F908CE2A3
:1010D00091E09F938F93BF920E941C030E94A104F2
:1010E000DC01CB018C010E944801812F992740E14E
:1010F000B7010E94BD07C6010E9405050F900F9021
:101100000F9086B399278D3F9105A1F08E3F9105F1
:1011100041F0AA2486B385BB8AE090E00E9448048F
:10112000B6CFAA20B9F7C85F8C2F99270E94050572
:10113000AB2CF0CFAA2071F7C850F6CFEF92FF92F8
:101140000F931F937B018C0120E030E040E05FE4CF
:101150000E946A0D88239CF020E030E040E05FECC4
:10116000C801B7010E94130ADC01CB01BC01CD010B
:101170000E94540E605070408040904804C0C801E6
:10118000B7010E94540E1F910F91FF90EF900895A8
:10119000A0E0B0E0EEECF8E00C943411FC014B015F
:1011A000BA0180E090E04081423008F481E000978D
:1011B000E1F4D4015C91523010F481E090E00097AA
:1011C00009F040C09C01443009F424C121153105C7
:1011D00089F0543061F0892B41F09181E4018981DB
:1011E000981719F040E750E018C1AF0116C181E02F
:1011F00090E0F1CFC901543009F409C1009711F50D
:101200009C01523009F400C121153105A9F042308A
:1012100081F0892B51F328E0DB0101900D922A9592
:10122000E1F78181E40199818923FB018183AB018D
:10123000F4C081E090E0EDCFC901423009F4E1C093
:10124000892B11F0A401E9C0A280B380E401CA8017
:10125000DB802481358146815781EC80FD800E81C1
:101260001F81C5018C199D0997FF03C09095819539
:101270009F4F80970CF0B8C0CA14DB04CCF4C501B2
:101280008C199D096C010894C108D108D801C701C7
:1012900081709070A070B07016950795F794E794E0
:1012A000E82AF92A0A2B1B2BC114D10461F7650126
:1012B000AC14BD04A4F40894A11CB11CDA01C9014A
:1012C00081709070A070B0705695479537952795AE
:1012D000282B392B4A2B5B2BAC14BD0464F3918172
:1012E000E4018981981709F46EC0992309F466C056
:1012F000E21AF30A040B150BA801970157FD4DC024
:10130000FB011182A282B3822483358346835783F3
:10131000FB012481358146815781DA01C90101979A
:10132000A109B1098F5F9F4FAF4FBF43C0F4220F98
:10133000331F441F551FEB012C833D834E835F8376
:101340008A819B8101978A839B83DA01C901019776
:10135000A109B1098F5F9F4FAF4FBF4340F383E0B7
:10136000DB018C9357FF63CFDA01C901B695A795CE
:10137000979587952170307040705070822B932B19
:10138000A42BB52BEB018C839D83AE83BF838A8115
:101390009B8101968A839B834ACF81E0FB018183F5
:1013A000A282B38288279927DC01821B930BA40BAE
:1013B000B50B84839583A683B783AACF2E193F09E3
:1013C000400B510B9BCFEB019983AA82BB82DA01C0
:1013D000C9018E0D9F1DA01FB11F8C839D83AE83FD
:1013E000BF839C01AD01BBCFCA14DB0424F4EE24FF
:1013F000FF24870174CF560120E030E040E050E048
:101400006ECF81E090E01CCF21E030E0FDCE81E0A6
:1014100090E0F4CE21E030E0D9CECA01ECE0CDB7C7
:10142000DEB70C945011A0E2B0E0E9E1FAE00C94D0
:101430003C11DC01CB01898F9A8FAB8FBC8F2D8F34
:101440003E8F4F8F58A3BE016F5F7F4FCE014996ED
:101450000E949B0F8E01075F1F4FB801CE014D9672
:101460000E949B0FAE014F5E5F4FB801CE01019607
:101470000E94C8080E94B80EDC01CB01BC01CD015E
:10148000E4E0A0960C945811A0E2B0E0EAE4FAE09F
:101490000C943C11DC01CB01898F9A8FAB8FBC8FF0
:1014A0002D8F3E8F4F8F58A3BE016F5F7F4FCE01B0
:1014B00049960E949B0F8E01075F1F4FB801CE0116
:1014C0004D960E949B0F8A8591E089278A87AE01FD
:1014D0004F5E5F4FB801CE0101960E94C8080E947E
:1014E000B80EDC01CB01BC01CD01E4E0A0960C9468
:1014F0005811A0E2B0E0EFE7FAE00C943C11DC01F7
:10150000CB01898F9A8FAB8FBC8F2D8F3E8F4F8FE2
:1015100058A3BE016F5F7F4FCE0149960E949B0F7B
:101520008E01075F1F4FB801CE014D960E949B0FA1
:10153000AE014F5E5F4FB801CE0101960E94AA0A2C
:101540000E94B80EDC01CB01BC01CD01E4E0A09605
:101550000C945811A6E0B0E0E0EBFAE00C942E11E8
:101560008C0149835A83882499245401140125014C
:1015700080E090E0D8012C91223008F481E00097BF
:1015800099F4DB013C91323010F481E090E0009757
:1015900039F5AC01243009F426C141155105A9F0F3
:1015A000323081F0892B59F420E0F8019181FB0160
:1015B0008181981321E0F8012183A80117C140E738
:1015C00050E014C181E090E0EDCFCA01343009F45D
:1015D00007C1009799F0CA01223069F0892B79F789
:1015E00020E0F8019181FB018181981321E0FB014A
:1015F0002183AB01FBC081E090E0F0CF223009F401
:10160000ECC0009789F6323009F4E4C0892B41F729
:10161000F80184819581A681B7818B839C83AD83FA
:10162000BE83FB012481358146815781CC24DD2492
:101630007601BFE16B2E712C8B819C81AD81BE81C7
:1016400081709070A070B070892BC1F080E090E044
:10165000220E331E441E551E22163306440655061E
:1016600008F481E0AA2797FDA095BA2F8C0D9D1D47
:10167000AE1DBF1D880E991EAA1EBB1ECC0CDD1C04
:10168000EE1CFF1C57FF08C081E090E0A0E0B0E036
:10169000C82AD92AEA2AFB2A220F331F441F551FC2
:1016A0008B819C81AD81BE81B695A79597958795D5
:1016B0008B839C83AD83BE8308946108710877FE99
:1016C000BBCFF80122813381FB0182819381280FF6
:1016D000391FE981FA812283338340E0F801918147
:1016E000FB018181981341E0E981FA8141832E5FFA
:1016F0003F4F22833383B7FE1CC0C901019682830A
:101700009383D501C40181709070A070B070892B53
:1017100061F0569447943794279480E090E0A0E0DD
:10172000B0E8282A392A4A2A5B2AB694A7949794C3
:10173000879490E0891690E0990690E0A90690E4DD
:10174000B90610F5E981FA8182819381019782833C
:101750009383880C991CAA1CBB1C57FE08C081E00F
:1017600090E0A0E0B0E0882A992AAA2ABB2A220C9D
:10177000331C441C551C90E0891690E0990690E0BB
:10178000A90690E4B906F0F2D501C4018F779070F4
:10179000A070B07080349105A105B10559F0E981C0
:1017A000FA8184829582A682B78283E08083498110
:1017B0005A811CC087FC05C0211431044104510426
:1017C00071F380E490E0A0E0B0E0880E991EAA1EBC
:1017D000BB1EE5CF81E090E019CF81E090E011CF12
:1017E00081E090E0F6CE41E050E0D7CECA01E2E1E0
:1017F00026960C944A11A8E1B0E0E1E0FCE00C94DC
:101800003C11DC01CB01898B9A8BAB8BBC8B2D8B74
:101810003E8B4F8B588FBE016F5F7F4FCE0141963D
:101820000E949B0F8E01075F1F4FB801CE014596A6
:101830000E949B0FB801CE0101960E94290C0E94C4
:10184000B80EDC01CB01BC01CD01E4E068960C943C
:101850005811A0E0B0E0EFE2FCE00C943611FC017E
:10186000DB0180E090E04081423008F481E00097A5
:10187000E9F49C015C91523008F421E02115310516
:1018800011F0BD01A5C0818111969C911197892706
:101890008183C901443009F498C0009729F442308B
:1018A00009F490C0009739F0451711F0BF0190C0BE
:1018B00060E770E08DC09C01543009F480C02115B0
:1018C000310539F014821582168217828283938340
:1018D000EDCFC901523009F46FC0892B19F084E0B3
:1018E0008083E4CF6281738112968D919C911397CE
:1018F000681B790B6283738324813581468157810C
:101900001496ED90FD900D911C9117972E153F05A3
:101910004007510740F4220F331F441F551F6150E9
:1019200070406283738380E090E0A0E0B0E4AA247A
:10193000BB2465012E153F054007510740F0A82A3A
:10194000B92ACA2ADB2A2E193F09400B510BB6953A
:10195000A79597958795220F331F441F551F009712
:10196000A105B10539F7D601C5018F779070A07038
:10197000B07080349105A105B10529F0A482B5822B
:10198000C682D78293CFA7FE09C080E490E0A0E092
:10199000B0E0A80EB91ECA1EDB1EF0CF211531051E
:1019A0004105510559F3A0E4B0E0C0E0D0E0AA0E33
:1019B000BB1ECC1EDD1EE2CF81E090E08ECF21E089
:1019C00030E07DCF81E090E06DCF81E090E065CFA9
:1019D000CB01EAE0CDB7DEB70C945211A8E1B0E03C
:1019E000E4EFFCE00C943C11DC01CB01898B9A8B79
:1019F000AB8BBC8B2D8B3E8B4F8B588FBE016F5F9B
:101A00007F4FCE0141960E949B0F8E01075F1F4FB3
:101A1000B801CE0145960E949B0F20E030E08981FD
:101A2000823008F421E02115310539F489858230AE
:101A300010F421E030E0232B19F081E090E008C0A1
:101A4000B801CE0101960E941010992787FD90954C
:101A5000E4E068960C945811A8E1B0E0E2E3FDE000
:101A60000C943C11DC01CB01898B9A8BAB8BBC8B2A
:101A70002D8B3E8B4F8B588FBE016F5F7F4FCE01FA
:101A800041960E949B0F8E01075F1F4FB801CE0148
:101A900045960E949B0F20E030E08981823008F457
:101AA00021E02115310539F48985823010F421E0D7
:101AB00030E0232B19F08FEF9FEF08C0B801CE0163
:101AC00001960E941010992787FD9095E4E0689692
:101AD0000C945811A8E1B0E0E0E7FDE00C943C1153
:101AE000DC01CB01898B9A8BAB8BBC8B2D8B3E8B16
:101AF0004F8B588FBE016F5F7F4FCE0141960E9482
:101B00009B0F8E01075F1F4FB801CE0145960E94C3
:101B10009B0F20E030E08981823008F421E021151C
:101B2000310539F48985823010F421E030E0232B2F
:101B300019F08FEF9FEF08C0B801CE0101960E9407
:101B40001010992787FD9095E4E068960C94581141
:101B5000A8E1B0E0EEEAFDE00C943C11DC01CB0121
:101B6000898B9A8BAB8BBC8B2D8B3E8B4F8B588F7D
:101B7000BE016F5F7F4FCE0141960E949B0F8E0189
:101B8000075F1F4FB801CE0145960E949B0F20E0D2
:101B900030E08981823008F421E02115310539F4E3
:101BA0008985823010F421E030E0232B19F081E0A8
:101BB00090E008C0B801CE0101960E94101099274C
:101BC00087FD9095E4E068960C945811A8E0B0E089
:101BD000ECEEFDE00C943A119B01AC0183E08983AB
:101BE00079018A01EE2417FDE394FF2400271127D1
:101BF000EA82211531054105510539F482E08983D6
:101C0000CE0101960E94B80E4BC08EE190E08B830E
:101C10009C83EE2009F43FC0203080E0380780E04C
:101C2000480780E8580791F188279927DC01821B33
:101C3000930BA40BB50B8D839E83AF83B8872D8147
:101C40003E814F8158852030E0E03E07E0E04E07BE
:101C5000E0E45E07A8F66B817C81DA01C901880F98
:101C6000991FAA1FBB1F615070409C01AD018030BD
:101C7000E0E09E07E0E0AE07E0E4BE0770F36B83B0
:101C80007C838D839E83AF83B887BACF60E070E09A
:101C900080E09FEC05C02D833E834F835887CFCFD4
:101CA000E6E028960C945611ACE0B0E0EAE5FEE0E0
:101CB0000C943E11DC01CB0189879A87AB87BC87E6
:101CC000BE016F5F7F4FCE0109960E949B0F80E09F
:101CD00090E02981223009F444C0009771F4223049
:101CE00010F481E090E0009741F42430B9F1892BA1
:101CF00061F42B813C8137FF05C060E070E080E03B
:101D000090E032C02F3131056CF08A81882329F0B0
:101D100060E070E080E090E827C06FEF7FEF8FEF2A
:101D20009FE722C08EE190E0821B930B2D813E81C4
:101D30004F81588504C056954795379527958A95C4
:101D4000D2F78A81882339F05095409530952195B6
:101D50003F4F4F4F5F4FCA01B90106C081E090E08D
:101D6000C6CF81E090E0B9CFE2E02C960C945A11F6
:101D7000A4E0B0E0EEEBFEE00C943A11FC0124810B
:101D80003581468157818181E82EFF2400E010E0F3
:101D9000C8016081623008F481E0892B21F00FEFE7
:101DA00010E04061AAC0C801643009F4A3C0892BC7
:101DB00009F074C0C801623009F499C0892B09F098
:101DC0006FC0211531054105510509F496C0828186
:101DD00093816FEF823896070CF05DC062E87FEF69
:101DE000681B790B6A31710564F120E030E040E056
:101DF00050E0DA01C9018F779070A070B070803424
:101E00009105A105B105B1F0215C3F4F4F4F5F4FE8
:101E1000203080E0380780E0480780E4580710F061
:101E200001E010E097E056954795379527959A95EC
:101E3000D1F763C027FFECCF205C3F4F4F4F5F4F80
:101E4000E7CFF80181E090E0A0E0B0E0062E04C00A
:101E5000880F991FAA1FBB1F0A94D2F70197A109E7
:101E6000B10982239323A423B5230097A105B105CB
:101E700009F0E1E004C056954795379527956A9596
:101E8000D2F7CF01AA2797FDA095BA2F282B392B7F
:101E90004A2B5B2BAECF803891053CF00FEF10E062
:101EA00020E030E040E050E028C08C0101581F4F96
:101EB000DA01C9018F779070A070B07080349105FD
:101EC000A105B10569F0215C3F4F4F4F5F4F57FFB0
:101ED000A9CF56954795379527950F5F1F4FA2CFEE
:101EE00027FFF5CF205C3F4F4F4F5F4FF0CF81E092
:101EF00090E064CF81E090E05ACF29833A83902F1D
:101F0000979599279795842F8F77892B8B83169593
:101F100007959E2D979599279795802F8F77892BD9
:101F20008C8389819A81AB81BC81BC01CD01E6E0C3
:101F300024960C945611FC01DB01408151812281D1
:101F4000622F6F7770E0221F2227221F9381892F33
:101F5000880F822B282F3327991F9927991F1196B5
:101F60009C93119721153105B9F54115510561056E
:101F7000710519F482E08C9352C02E5730401296AE
:101F80002D933C931397E7E0440F551F661F771F6F
:101F9000EA95D1F783E08C934030F0E05F07F0E002
:101FA0006F07F0E47F0790F4C901440F551F661FC7
:101FB000771F0197403020E0520720E0620720E4BD
:101FC000720798F312968D939C931397FD014483A7
:101FD00055836683778323C02F3F310591F02F57B8
:101FE0003040FD0112962D933C93139783E08C9320
:101FF00087E0440F551F661F771F8A95D1F77064DD
:10200000E6CF411551056105710511F484E0B3CFA8
:1020100064FF03C081E08C93D9CF1C92D7CF089581
:10202000A0E0B0E0E6E1F0E10C943911FC01DB0145
:1020300080E090E04081423008F481E0009739F47C
:102040005C91523010F481E090E0009719F061E06B
:1020500070E08EC09C01443009F487C0232B69F0E6
:10206000543009F47FC0892B41F011968C91682F70
:1020700077278181681B71097BC080E090E0443044
:1020800009F46DC0009749F5543009F465C0009714
:10209000A1F49C01423009F45CC0232B39F09C016F
:1020A000523009F453C0232B09F047C080E090E080
:1020B000423009F448C0009759F011968C9188235A
:1020C00021F48FEF9FEFBC0153C081E090E0FBCF84
:1020D0009C015230A9F1232B21F08181882389F7BB
:1020E000F4CFD18011968C911197D81619F0DD207C
:1020F00041F7EBCF4281538112968D919C911397BA
:1021000084179507A4F348175907A4F0E480F580D5
:102110000681178114964D915D916D917C91179771
:102120004E155F056007710710F3E416F506060704
:10213000170718F4DD2029F2C8CF60E070E018C05E
:1021400021E030E0C8CF81E090E0B5CF21E030E081
:10215000AACF21E030E0A1CF81E090E098CF81E0EC
:1021600090E090CF81E090E07ECF21E030E076CF2C
:10217000CB01E7E0CDB7DEB70C945511629FD001DB
:10218000739FF001829FE00DF11D649FE00DF11D32
:10219000929FF00D839FF00D749FF00D659FF00DE1
:1021A0009927729FB00DE11DF91F639FB00DE11DCE
:1021B000F91FBD01CF0111240895AA1BBB1B51E1DA
:1021C00007C0AA1FBB1FA617B70710F0A61BB70BA7
:1021D000881F991F5A95A9F780959095BC01CD014C
:1021E0000895A1E21A2EAA1BBB1BFD010DC0AA1F58
:1021F000BB1FEE1FFF1FA217B307E407F50720F070
:10220000A21BB30BE40BF50B661F771F881F991FEA
:102210001A9469F760957095809590959B01AC0133
:10222000BD01CF01089597FB092E05260ED057FD5D
:1022300004D0D7DF0AD0001C38F450954095309573
:1022400021953F4F4F4F5F4F0895F6F7909580953A
:10225000709561957F4F8F4F9F4F08952F923F92BA
:102260004F925F926F927F928F929F92AF92BF92A6
:10227000CF92DF92EF92FF920F931F93CF93DF9352
:10228000CDB7DEB7CA1BDB0B0FB6F894DEBF0FBEAF
:10229000CDBF09942A88398848885F846E847D84FC
:1022A0008C849B84AA84B984C884DF80EE80FD80FE
:1022B0000C811B81AA81B981CE0FD11D0FB6F89474
:0C22C000DEBF0FBECDBFED010895FFCFC3
:00000001FF
